:100000000C9427020C945F020C945F020C945F0224
:100010000C945F020C945F020C945F020C945F02DC
:100020000C945F020C945F020C94A41D0C94761E39
:100030000C94F8170C945F020C945F020C945F020E
:100040000C945F020C945F020C945F020C945F02AC
:100050000C945F020C9480180C945F020C945F0265
:100060000C945F020C945F020C945F020C945F028C
:100070000C945F020C945F020C945F020C945F027C
:100080000C945F020C945F020C945F020C945F026C
:100090000C945F020C945F020C945F020C945F025C
:1000A0000C945F020C945F020C945F0242064206BD
:1000B0006E066E06D606010801080108F4068D07D3
:1000C0009E079E07E31E0A1F02200A1F0220561FDA
:1000D000791F0220D01FDF1F29003A003B003C009F
:1000E0003D003E003F00400041004200430044000C
:1000F0004500310046004700480035001E001F0043
:1001000020002100220023002400250026002700D3
:100110002D002E002A0049004A004B002B0014003D
:100120001A000800150017001C0018000C0012002F
:1001300013002F00300031004C004D004E003900FC
:1001400004001600070009000A000B000D000E0055
:100150000F003300340031002800000000000000D0
:10016000E10064001D001B000600190005001100DD
:100170001000360037003800E50001510000520041
:100180000000E000E300E2000000000000002C009E
:100190000000000000000000E600E700E40050005E
:1001A00051004F00010001000100010001000100A9
:1001B0000100010001000100010001000100010037
:1001C0000100010001000100010001000100010027
:1001D0000100010001000100010001000100010017
:1001E0000100AA00A800A90001000100010001000F
:1001F00001000100010001000100010001000100F7
:1002000001000100AC00AE00AB00010001000100E4
:1002100001000100010001000100010001000100D6
:1002200001000100010000000000000001000100C9
:1002300001000100010001000100010001000100B6
:1002400001000100010001000000010000000100A8
:10025000010001000000000000000100000000009B
:100260000000000001000100010001000100010088
:1002700044454255473A2064697361626C65642E57
:100280000A0044454255473A20656E61626C6564D8
:100290002E0A000A0025303258006C65645F7461D4
:1002A000736B3A20004F6E6573686F743A20616318
:1002B000746976653A2025640A000A0025303332D5
:1002C0006C62003A200025303258000A722F6320F9
:1002D000303132333435363738394142434445467C
:1002E000303132333435363738394142434445466C
:1002F0000A000A002530325820006B6579626F6170
:1003000072645F7265706F72743A20005B735D0097
:100310005B575D005B535D005B525D005B445D00BD
:100320005B435D0012034F006D0072006F006E00B2
:1003300054004B004C0000000E034500760079008D
:1003400064003100330000000403090409025B006B
:10035000030100A0FA0904000001030101000921C2
:100360001101000122400007058103080001090472
:1003700001000103000000092111010001223200E7
:1003800007058203200001090402000203000000A7
:100390000921110100012222000705830320000129
:1003A00007050303200001120100020000000805F8
:1003B0004778EA0100010200010631FF0974A1013A
:1003C0000975150026FF009520750881020976152C
:1003D0000026FF00952075089102C005010980A143
:1003E00001850319012AB700150126B7009501758B
:1003F000108100C0050C0901A101850419012AA082
:1004000002150126A002950175108100C0050109A1
:1004100006A101050719E029E715002501950875D2
:100420000181029501750881010507190029FF1551
:100430000026FF00950675088100050819012905A9
:10044000950575019102950175039101C000112474
:100450001FBECFEFDAE0DEBFCDBF04B603FE18C08B
:100460008091B6029091B702A091B802B091B90202
:100470008730904BA740B04B59F41092B6021092BF
:10048000B7021092B8021092B902E0E0F8E30995C1
:1004900011E0A0E0B1E0E0E3F1E402C005900D92CC
:1004A000AA39B107D9F722E0AAE9B1E001C01D924B
:1004B000A63BB207E1F70E9498140C9496200C9486
:1004C0000000FF93EF93E0919A01F0919B01309728
:1004D00009F00995EF91FF910895FC018591803015
:1004E00011F0EFDFFBCF0895FF27E0E230E247FF96
:1004F0000CC0419597FF09C0EDE26095709580951D
:100500009095611D711D811D911D27FF02C02195D0
:1005100030E350E2AA27660F771F881F991FAA1F92
:10052000A41710F0A41B63955A95A9F7AA3008F0F8
:10053000A95FA05DAF93F3956115710581059105E4
:1005400041F7ED3211F4EF93F395F21718F43F935E
:10055000F395FBCF8F91B5DFFA95E1F70895E99117
:10056000F9918591803021F0853219F0AADFF9CF19
:10057000089520E0E89455915532C1F3503311F4B9
:10058000689455915A3348F4505390F3220F022E39
:10059000220F220F200D250FF4CF0EF42195899103
:1005A0009991533619F3533729F1533559F1BC0159
:1005B00088279927E8945C3621F489919991689469
:1005C0005591543639F446EF7EF077FF0DC08FEF2A
:1005D0009FEF0AC055374AE039F0583540E121F025
:1005E000523642E009F00895FF93EF937DDFEF91DB
:1005F000FF91B7CFFF93EF93FC0181918030B9F366
:1006000060DFFBCFFF93EF9368DFF1CFDF93CF93F2
:10061000CDB7DEB72596A3DFCF91DF91089581E0B6
:10062000089581E008950C94110308950C94150326
:100630001F93CF93DF9300D000D01F92CDB7DEB7CA
:1006400049835A836B8330919D0189819A8131114D
:1006500014C0662359F0222349F00E943A0A182F49
:10066000682F89819A810E94E30903C00E940E0AC3
:10067000182F69817A81812F04C00E943A0A69810A
:100680007A810F900F900F900F900F90DF91CF9184
:100690001F910C949A11FC01262F40815181628197
:1006A000738184810C94180381E00895CF93DF93C4
:1006B000EC0160E00E944B03BE01DF91CF910C94EE
:1006C00016030C942B130C94271308950E948D0885
:1006D0000E9465032FEF84E39CE02150804090400E
:1006E000E1F700C000000C94A6180F931F93CF935E
:1006F000DF938C0161E00E944B03EC01B8010E9482
:100700001303882309F45BC0B801CE010E9491163F
:10071000882309F454C0B801CE010E94A51488238F
:1007200009F44DC0B801CE010E94ED15882309F4EB
:1007300046C0F80182818823D9F1CF3D8CE5D807E6
:1007400079F140F4C115FCE5DF0791F0C130DC45DB
:1007500091F02EC0CC35EDE5DE0741F1CD35FDE55C
:10076000DF0709F1CB35DD4519F50E94D10E20C018
:100770000E94660324C080915302C82FC095C170A7
:10078000C0FB80F980935302CC2329F082E892E0E9
:100790000E946D0214C080E792E00E946D0210C0BA
:1007A0000E94850F0CC00E94C80E02C00E94D40E89
:1007B000C801DF91CF911F910F910C940F03C0E0FE
:1007C0008C2FDF91CF911F910F9108950E94D81720
:1007D0000C944F040E9452040C94DE178295982FBB
:1007E000937344E0949F900111248C7C86958695A8
:1007F000282B822F8575880F2A7A2695822B0895BB
:10080000CF93DF93D92F0E94EE03C82F8D2F0E9424
:10081000EE032C2F30E0322F2227A901482BCA01EA
:10082000DF91CF910895CF92DF92EF92FF920F93D5
:100830001F93CF93DF936B017C01CB010E940004D7
:10084000EC01C7010E940004AC01CE01A0E0B0E0C1
:10085000DC019927882760E070E08C019D01042B62
:10086000152B262B372BC901B801DF91CF911F9192
:100870000F91FF90EF90DF90CF90089508950C9422
:100880003E0481E008950C9441040895CF93C82F4D
:100890000E943F048C2F0E944304CF91089580E072
:1008A0000C9446040E94ED160C944604CF930E94CB
:1008B000ED16C82F80919C01C81741F1C0939C018F
:1008C0008091530282FF1EC080FF04C08AE992E03B
:1008D0000E946D028091530280FF0CC01F92CF9343
:1008E00085E992E09F938F930E9406030F900F90EB
:1008F0000F900F908091530280FF04C083E992E033
:100900000E946D028C2FCF910C944604CF910895D4
:10091000CF93DF93CDB7DEB72B970FB6F894DEBF3A
:100920000FBECDBF4F83588769877A878B87611148
:100930000E94000E9E012F5F3F4F86E0F901119249
:100940008A95E9F785E0FE013796D90101900D926D
:100950008A95E1F789819A814C815D81452B31F03F
:100960009F3F31F491E08F3F19F403C091E001C043
:1009700090E090FF09C049815A816B817C818D8113
:100980009E810E94210D05C0C9010E94540381115E
:10099000F2CF2B960FB6F894DEBF0FBECDBFDF911E
:1009A000CF910895FC01808191810E947C0A089575
:1009B000CF93882309F49CC0C82F8238C1F40E94C9
:1009C000ED1681FD95C069E38091020190910301CC
:1009D0000E94B0170E94220E2FEF81EE94E021506A
:1009E00080409040E1F700C0000069E319C08338FF
:1009F00001F50E94ED1680FD7BC063E58091020148
:100A0000909103010E94B0170E94220E2FEF81EEF9
:100A100094E0215080409040E1F700C0000063E581
:100A200080910201909103010E94B217CF910C9422
:100A3000220E8438C1F40E94ED1682FD59C067E48D
:100A400080910201909103010E94B0170E94220E32
:100A50002FEF81EE94E0215080409040E1F700C0FC
:100A6000000067E4DDCF8CEF8C0F813AD0F46C2F5F
:100A700080910201909103010E947A17882349F026
:100A80006C2F80910201909103010E94B2170E9485
:100A9000220E6C2F80910201909103010E94B017E9
:100AA000C5CF80E28C0F883048F4C77081E001C068
:100AB000880FCA95EAF70E94E30DB8CFEBE5EC0F7B
:100AC000E33040F4F0E0E15CFE4F808190E0CF91B4
:100AD0000C944217C85AC73158F4EC2FF0E0EE0FCF
:100AE000FF1FEF5EFE4F80819181CF910C945817CC
:100AF000CF910895882309F45BC0682F823879F478
:100B00000E94ED1681FF54C069E38091020190912B
:100B100003010E94B0170E94220E69E310C08338BF
:100B2000B1F40E94ED1680FF43C063E5809102019D
:100B3000909103010E94B0170E94220E63E58091FC
:100B40000201909103010E94B2170C94220E843886
:100B500079F40E94ED1682FF2BC067E480910201B8
:100B6000909103010E94B0170E94220E67E4E7CF24
:100B70008CEF860F813A18F380E2860F883048F4B4
:100B8000677081E001C0880F6A95EAF70E94E90D5D
:100B9000DCCF8BE5860F833020F480E090E00C946E
:100BA0004217685A673120F480E090E00C9458179F
:100BB00008951F93CF93DF93182FEB010E94D80461
:100BC000209741F08FE99FE00197F1F700C0000006
:100BD0002197F6CF812FDF91CF911F910C947A0549
:100BE000893319F060E070E002C060E570E00C94B9
:100BF000D905882321F00E94E30D0C94220E08955C
:100C0000882321F00E94E90D0C94220E0895CF92C2
:100C1000DF92EF92FF920F931F93CF93DF937C01AC
:100C2000D62FC72FFC011281058102950F700E94FB
:100C3000D90D8823B9F01123A9F08C2F807F80343F
:100C400021F080E28D0F883068F08091740282FD7F
:100C500009C082E00E94820E0E94D90D91E0D82E38
:100C6000D92601C0D12CCC2EC2948FE0C8228C2D65
:100C700090E08C30910508F0C4C1FC01EA5AFF4FA6
:100C80000C9441208C2F807FCF70882311F0C29567
:100C9000C07F112399F0CC2309F49FC180E28D0F0E
:100CA000883010F0D11104C08C2F0E94E30D03C0D6
:100CB0008C2F0E94F30D0E94220E8FC18D2F0E9457
:100CC0007A05CC2309F49DC180E28D0F883038F17C
:100CD000DD2329F18C2F0E94F90D24C08C2F807FF9
:100CE000CF70803211F0C295C07FDD2319F0D13072
:100CF000A1F13DC08091740282FF17C0112349F019
:100D0000CC2329F08C2F0E94E30D0E94220E80E05C
:100D100065C180E00E947A05CC2309F472C18C2F52
:100D20000E94E90D0E94220E6CC1112371F0002374
:100D300041F0013031F40E94030E8C2B0E940B0E07
:100D400060C10E94030E8C2B1DC0002319F00130DE
:100D500009F457C10E94180E25C0112321F0063056
:100D600008F04FC10EC0053008F04BC11BC0112365
:100D700061F0002331F0F701858180FF2EC18F7073
:100D800085838C2F0E94F9053CC1002359F0D9338B
:100D900009F034C1FFEF07EE13E0F15000401040BE
:100DA000E1F72AC18C2F0E9400062BC18C2F86955B
:100DB0008695837019F0813061F023C1112321F0F1
:100DC0008D2F9C2F937002C080E090E00E9442170C
:100DD00020C1112321F08D2F9C2F937002C080E041
:100DE00090E00E94581715C18C2F837009F047C0FE
:100DF00011110BC12D2F229526952770220F220F3E
:100E00006D2F6F70862F90E0A0E0B0E0022E04C03E
:100E1000880F991FAA1FBB1F0A94D2F7D4FF10C0D6
:100E20004FE050E060E070E004C0440F551F661FC3
:100E3000771F2A95D2F7409550956095709503C01D
:100E400040E050E0BA01C695C695C3708A019B0187
:100E5000082B192B2A2B3B2BC901B801C23049F0B2
:100E600058F4C13019F00E94F908CFC00E94E70879
:100E7000CCC00E940B09C9C00E94E508C6C011235E
:100E800019F08C2F817001C08695882309F4BDC0AC
:100E90002D2F229526952770220F220F6D2F6F7010
:100EA000862F90E0A0E0B0E0022E04C0880F991FCA
:100EB000AA1FBB1F0A94D2F7D4FF10C04FE050E026
:100EC00060E070E004C0440F551F661F771F2A952D
:100ED000D2F7409550956095709503C040E050E082
:100EE000BA01C695C695C3708A019B01082B192BC0
:100EF0002A2B3B2BC901B801C23049F058F4C1304C
:100F000019F00E94BE0981C00E94AC097EC00E94F7
:100F1000D0097BC00E941F0978C0CF70112339F01F
:100F20008C2F0E9445098D2F0E94F9056EC08D2FD0
:100F30000E9400068C2F0E94660967C0D23F21F1F3
:100F400028F4D03F41F0D13FC1F043C0D33F19F165
:100F5000D43F79F03EC0112341F0053008F051C074
:100F60008C2F8F710E948B094CC0063008F049C04D
:100F7000F7CF8091740282FF18C0112339F08C2FB3
:100F80008F710E9445093DC01123C9F38C2F8F71C9
:100F90000E94660936C0112329F08C2F8F710E94A0
:100FA00030092FC00E942B092CC0112349F0CF71AA
:100FB0008C2F0E94450963E08C2F0E94670E21C090
:100FC00081E00E94820E0230E0F082E00E94820EF8
:100FD00018C0112331F0002391F28D2F0E94D80404
:100FE00010C0002399F2D93349F41FEF27EE33E004
:100FF000115020403040E1F700C000008D2F0E94CA
:101000007A0588EF8C0D843020F40E94ED160E9442
:101010004604DD20C9F00E94D50D80FD15C0F70102
:1010200012820E94CF0D0E944509C7010E94450807
:101030000E94CF0DDF91CF911F910F91FF90EF9004
:10104000DF90CF900C946609DF91CF911F910F91A3
:10105000FF90EF90DF90CF9008950F931F93CF9361
:10106000DF93EC01688179818A810E94870A8C0173
:101070000E94E2090E94D308B801CE010E9407062F
:10108000DF91CF911F910F910895CF93DF93EC01E2
:10109000988189812B813C81232B31F08F3F31F462
:1010A00081E09F3F19F403C081E001C080E080FD32
:1010B0001DC0CE010E947503811110C00E94D90D80
:1010C0008823A1F08A81882389F08091740282FDAF
:1010D0000DC082E0DF91CF910C94820ECE010E9470
:1010E0002D08CE01DF91CF910C945603DF91CF9163
:1010F000089580E090E00E94421780E090E00E9416
:1011000058170E94000E0C94220E809102019091BB
:1011100003010E94B4170C9479080E94F00D0C94FE
:10112000850892959F70963079F010F4925001C026
:101130009A50923068F4803F69F018F4883E40F489
:1011400009C0843F29F406C0883E20F0813F11F099
:1011500080E0089581E00895FC01808191810E94E2
:101160007C0A0E9491080895CF93DF9300D000D0AD
:101170001F92CDB7DEB70F900F900F900F900F908A
:10118000DF91CF910895CF93DF9300D000D000D0AE
:10119000CDB7DEB726960FB6F894DEBF0FBECDBF33
:1011A000DF91CF910895089508950C94D4080C947C
:1011B000D5080E94D7086093E3017093E4018093FF
:1011C000E5019093E6010C9479080C94D9080F93EB
:1011D0001F930091E3011091E4012091E50130910A
:1011E000E601602B712B822B932B1F910F910C9496
:1011F000D9080F931F930091E3011091E40120910E
:10120000E5013091E60160237123822393231F912E
:101210000F910C94D9080F931F930091E301109143
:10122000E4012091E5013091E601602771278227D2
:1012300093271F910F910C94D9080C94D4080E9405
:101240001D096093DF017093E0018093E1019093A9
:10125000E2010C94790860E070E0CB010C941F0966
:101260000F931F9341E050E060E070E08A019B0122
:1012700004C0000F111F221F331F8A95D2F7C90126
:10128000B8011F910F910C941F090F931F9341E018
:1012900050E060E070E004C0440F551F661F771FE8
:1012A0008A95D2F78091DF019091E001A091E10150
:1012B000B091E2018A019B01082B192B2A2B3B2BB1
:1012C000C901B8011F910F910C941F090F931F932F
:1012D00041E050E060E070E004C0440F551F661F1D
:1012E000771F8A95D2F740955095609570958091BB
:1012F000DF019091E001A091E101B091E2018A014A
:101300009B01082319232A233B23C901B8011F91FC
:101310000F910C941F090F931F9341E050E060E080
:1013200070E004C0440F551F661F771F8A95D2F7DF
:101330008091DF019091E001A091E101B091E20183
:101340008A019B01082719272A273B27C901B801D1
:101350001F910F910C941F090F931F930091DF01B0
:101360001091E0012091E1013091E201602B712B9D
:10137000822B932B1F910F910C941F090F931F9396
:101380000091DF011091E0012091E1013091E20133
:1013900060237123822393231F910F910C941F09C3
:1013A0000F931F930091DF011091E0012091E10163
:1013B0003091E20160277127822793271F910F91B7
:1013C0000C941F09089521E1929F800D1124E82FAC
:1013D000E695E695E695877051E001C0550F8A9530
:1013E000EAF785E0E89FF0011124E256FE4F20E085
:1013F00030E070E04081CB01022E02C096958795C7
:101400000A94E2F78170819584278523842781934C
:101410002F5F3F4F2530310569F7089521E1929FF5
:10142000800D1124682F669566956695982F9770A4
:1014300085E0689FB001112440E050E080E0FB01AE
:10144000E40FF51FE256FE4F208130E0092E02C066
:10145000369527950A94E2F721703327042E01C0B0
:10146000220F0A94EAF7822B4F5F5F4F45305105F8
:1014700031F70895BF92CF92DF92EF92FF920F93D0
:101480001F93CF93DF938C01C090DF01D090E001D8
:10149000E090E101F090E2018091E3019091E4019C
:1014A000A091E501B091E601C82AD92AEA2AFB2ACF
:1014B000CFE1D0E0D701C6010C2E04C0B695A795A8
:1014C000979587950A94D2F780FD04C0219790F7ED
:1014D000B12C07C0BC2EB8018C2F0E94AD11019712
:1014E000A9F38B2DDF91CF911F910F91FF90EF907A
:1014F000DF90CF90BF900895CF93DF93EC010E94CF
:101500003A0ABE010E94AD11DF91CF9108951F9359
:10151000CF93DF93EB0190919D01992321F0CB01B3
:101520000E947C0A13C0882349F0CB010E943A0A2A
:10153000182F682FCE010E94E30904C0CB010E943E
:101540000E0A182FBE01812F0E94AD11DF91CF919D
:101550001F9108951F93CF93DF93C091E70116E089
:101560008091E801C81799F0D0E01C9FF0011D9F01
:10157000F00D1124E751FE4F40815181628173814A
:10158000848195810E94C3082196C770E9CFDF91BD
:10159000CF911F9108954091190250911A026091C4
:1015A0001B0270911C0280911D0290911E020C94EE
:1015B000C308EF92FF920F931F93CF93DF93809115
:1015C0001E0282958F7009F065C080911B028823EE
:1015D00009F460C08091E701F090E80110911902D0
:1015E00000911A0260911C0270911D0291E01F3F50
:1015F00009F090E0C0910001D0910101292F96E0FF
:10160000E92E8F1509F446C06115710521F00F3FD1
:1016100021F030E003C031E001C0322F90E030FD16
:1016200036C0E89EF001E99EF00D1124DF01A751BC
:10163000BE4F11963C911197301329C03C91311344
:1016400026C012963C911297311121C013964D91EC
:101650005C911497461B570B4C175D07C0F48091A3
:101660001E028F70806180931E02E251FE4F8081C6
:101670008F708061808389E192E00E944508DF914C
:10168000CF911F910F91FF90EF900C94AA0A0196B1
:101690008770B7CFDF91CF911F910F91FF90EF909F
:1016A00008959F92AF92BF92CF92DF92EF92FF92F6
:1016B0000F931F93CF93DF93CDB7DEB761970FB62C
:1016C000F894DEBF0FBECDBF8C0185E0F801DE01CE
:1016D0001D9601900D928A95E1F7D8011296EC9033
:1016E00090911902E0911A0220911C0230911D0282
:1016F0002115310531F0EF3F31F481E09F3F19F4BE
:1017000003C081E001C080E0B82FB1709B2E80FD46
:1017100047C1D8014C9111965C9111971396AD90E9
:10172000BC90149789E1C82E82E0D82EF0901B025D
:10173000B501621B730B2091000130910101FF2064
:1017400009F4D9C080911E026217730708F095C092
:10175000282F207F09F052C05E1313C0491311C017
:10176000FE2CE1100EC08F70806180931E020E94DB
:10177000CB0AC6010E94450880911E02F8018583AC
:101780004DC1AB2831F05F3F31F481E04F3F19F498
:1017900003C081E001C080E080FD03C081E08E25B0
:1017A00002C080E090E0F82FF170FF2E80FF1CC097
:1017B0008091E7012091E80136E0821709F40BC11E
:1017C00090E0389FF001399FF00D1124E751FE4F52
:1017D0006181561306C06081461303C06281E61220
:1017E00003C001968770E9CFFE2CEE2009F416C1E4
:1017F00080911E02816080931E0254C05E1306C059
:10180000491304C0E11002C0F80199C0C8010E9448
:10181000AC08882361F1EE2051F120911E02822F45
:1018200082958F7090E0029774F0809119029091E8
:101830001A0298878F831986BB86AA862C87CE01C9
:1018400007960E94450886E0F801A9E1B2E0019000
:101850000D928A95E1F70E94D90A0E94CB0A0AC02C
:101860005E1711F1C8010E94AC0881112CC0C8019B
:101870000E944508FF24F394D1C0282F207F81F7D0
:101880007A2DB98AA88A6E2D89890E94B40889E1C7
:1018900092E00E94450886E0D6011D928A95E9F7FC
:1018A0000E94CB0AF12CBAC04913DCCFE110DACF89
:1018B000F8018583C8010E94450886E0D6011D9283
:1018C0008A95E9F7ABC0EE2091F220911E02822F9B
:1018D00082958F7090E002970CF4B5CF8091190239
:1018E00090911A029A8389831B82BD82AC822E83D7
:1018F000CE010196A6CF6217730708F044C0FE2CF4
:10190000EE2009F4B4CF5E1330C049132EC02091ED
:101910001E0220FD21C0822F82958F70482F50E03B
:1019200041155105C9F0F80125834F30510541F0AB
:101930008F5F982F9295907F822F8F70892B858350
:10194000C8010E94450886E0F801A9E1B2E00190D3
:101950000D928A95E1F73CC086E0F801A9E1B2E07A
:1019600001900D928A95E1F759C0C8010E94AC0818
:10197000811169CF80911E02816080931E02C8018F
:101980000E9445084BC07A2DB98AA88A6E2D898994
:101990000E94B40886E0D6011D928A95E9F718C026
:1019A000EE2009F464CFC8010E94AC08F82E882309
:1019B00009F45DCF86E0F801A9E1B2E001900D9253
:1019C0008A95E1F789E192E00E94D2040E94D90A47
:1019D0000E94CB0A23C04D875E878D859E850E941D
:1019E0007C0A292F22952F70223028F49F7039F01D
:1019F000811105C00BC0243028F49F7049F4805E2B
:101A0000883020F0C8010E9445089F2CF92C06C0A0
:101A1000D80115969C91907F91F7F8CF8F2D619604
:101A20000FB6F894DEBF0FBECDBFDF91CF911F91EF
:101A30000F91FF90EF90DF90CF90BF90AF909F906D
:101A400008951F93CF93DF93CDB7DEB72C970FB6D2
:101A5000F894DEBF0FBECDBF4F83588769877A8762
:101A60008B879C87CE0107960E94510B8823D1F06B
:101A70009F8188852A853B85232B31F08F3F31F468
:101A800081E09F3F19F403C081E001C080E080FD48
:101A900047C04F81588569857A858B859C850E94D2
:101AA000C3083EC086E0FE013796DE011196019024
:101AB0000D928A95E1F7FF81E8856A857B8561153E
:101AC000710531F0EF3F31F481E0FF3F19F403C0BD
:101AD00081E001C080E080FD23C02091E80130E07A
:101AE000C9010196877099274091E70150E084175A
:101AF0009507F1F1F983EA837D836C8396E0929FE9
:101B0000D001939FB00D1124A751BE4FFE01319615
:101B100001900D929A95E1F78093E8010E94AA0A3C
:101B200016E08091E7019091E801891771F1189F03
:101B3000C001112487519E4F0E94510B882329F127
:101B4000E091E7011E9FF0011124E751FE4F408113
:101B5000518162817381848195810E94C308809143
:101B6000E70190E00196877099278093E701D9CF2C
:101B70000E948D081092E8011092E701E9E1F2E07D
:101B800086E0DF011D928A95E9F72C960FB6F8944E
:101B9000DEBF0FBECDBFDF91CF911F910895809121
:101BA00027028595859585950895809127028770F0
:101BB000089590912702977081E009F480E00895DC
:101BC00080913202089590913202892B80933202E3
:101BD000089580959091320289238093320208956E
:101BE00010923202089590913102892B8093310234
:101BF0000895809590913102892380933102089550
:101C000010923102089580912802089508950C944D
:101C1000060E0C94070E9091740292FD08C09091EC
:101C20002802981721F0809328020C94090E089539
:101C300080912802882329F01092280280E00C94D9
:101C4000090E0895CF93DF93E0910201F091030113
:101C5000809132028083E0910201F0910301908132
:101C600080913102892B808380912802882381F022
:101C7000E0910201F09103019081892B8083809192
:101C80000201909103010E946E1781110E94180EAB
:101C9000C0910201D091030148E050E06FE172E091
:101CA000CE010E944720892B69F088E0FE01AFE158
:101CB000B2E001900D928A95E1F7CE01DF91CF91CC
:101CC0000C94F916DF91CF9108950C94060E909123
:101CD000740292FD10C098E0899F90011124262B78
:101CE000209327020E9445098091270285958595BA
:101CF00085950C94650E0C9445091092270280E09E
:101D00000C94650E209127028095822380932702F0
:101D1000982F977099F430E0482F082E000C550B3F
:101D20002417350759F09091740292FD07C08595EC
:101D3000859585950E9466090C947D0E0895CF9334
:101D40009091740292FB222720F92817F9F0C82FEE
:101D5000892FC0FB82F98093740280917302909165
:101D600074020E94010F82E00E94820E8091530251
:101D700080FF0CC01F92CF9385EA92E09F938F93D0
:101D80000E9406030F900F900F900F90CF9108952F
:101D90008091740282FB882780F991E089270C9456
:101DA0009F0E81E00C949F0E80E00C949F0E6FEFCD
:101DB0007FEF80E090E00C94802080E090E00E9433
:101DC0005C2021E0893E9E4F09F020E0822F08959B
:101DD00082E090E00C94542083E090E00C94542036
:101DE000CF9384E090E00E945420C82F82E290E0DC
:101DF0000E9454202C2F30E0A901582BCA01CF910A
:101E00000895CF93C92F682F84E090E00E9462204C
:101E10006C2F82E290E0CF910C946220AB01BC0168
:101E20008FE090E00C947420AB01BC0183E190E062
:101E30000C94742060E070E0CB010C94140F60E00F
:101E400070E0CB010E940E0F0C941A0F69EE7EEF2A
:101E500080E090E00E94802060E082E090E00E94BC
:101E6000622060E083E090E00E9462201092E30133
:101E70001092E4011092E5011092E60160E084E026
:101E800090E00E94622060E082E290E00E94622086
:101E900060E085E090E00E94622060E086E090E0F3
:101EA0000E9462206FEF87E090E00E94622040E095
:101EB00050E0BA0188E090E00E94742060E08DE07C
:101EC00090E00E94622040E050E0BA0188E190E09A
:101ED0000E94742060E087E190E00E94622040E070
:101EE00050E0BA018CE190E00E94742060E070E064
:101EF00080E290E00E94802040E050E0BA0188E15A
:101F000090E00E9474200C941F0F0C94260F682FF1
:101F10008EE090E00C9462200E94651860934F025E
:101F200070935002809351029093520260934B023F
:101F300070934C0280934D0290934E02089585B7A2
:101F4000806885BF85B7806885BF089581E0089562
:101F50000C94A60F08950C94AA0F0C94AA0F0C943D
:101F6000AD0F0C94AA0F0C94B10F0C94AA0F0E9401
:101F70009F0F8FE79AE10E94E3160E94B50F0C9421
:101F8000B30F0E94AB0F0C94AA0F0E94A1120C94E5
:101F900045040E9450180E94EF130E94C50F0C9434
:101FA000AF0F2F923F924F925F926F927F928F92DC
:101FB0009F92AF92BF92CF92DF92EF92FF920F93D8
:101FC0001F93CF93DF93CDB7DEB72D970FB6F8945D
:101FD000DEBF0FBECDBF0E940414282E81110E94C7
:101FE0008C0F83E392E09D878C8700E010E0302E19
:101FF000802F0E94C5122B013C01EC85FD8581914B
:102000009191A191B191FD87EC87530142018826FE
:102010009926AA26BB2681149104A104B104B1F427
:102020000F5F1F4F0630110511F78FEF89838A83E9
:102030001B820E9459188160782F9D838C8349816F
:102040005A816B818D810E94880451C08091530216
:1020500081FD0E94D1121B86C12CD12C7601C39424
:10206000D501C4018C219D21AE21BF21892B8A2B52
:102070008B2B91F10E94A80F8823D1F0FB85FE8362
:102080003F824C205D206E207F2081E0452846283D
:10209000472809F480E088870E9459188160782FCA
:1020A0009A8789874E815F8168858A850E94880426
:1020B000000F111F000F111FF801ED5CFD4F808113
:1020C0009181A281B381C826D926EA26FB26C08247
:1020D000D182E282F3820BC08B858F5F8B87CC0C21
:1020E000DD1CEE1CFF1C813109F0BACF99CF81E0D5
:1020F000211001C080E02D960FB6F894DEBF0FBE10
:10210000CDBFDF91CF911F910F91FF90EF90DF90A6
:10211000CF90BF90AF909F908F907F906F905F9087
:102120004F903F902F9008950E94D10F0C94560429
:10213000CF93DF930E94B211EC01811522E5920743
:10214000E8F5811531E5930708F0B6C0883E9105A2
:1021500028F5803E910508F0E9C0883A910570F4B1
:10216000853A910508F07AC08130910509F473C071
:1021700008F4D9C0049708F0D9C0D5C08F3B9105A9
:1021800008F0D1C0C85AD0E0CC0FDD1FCE5BDE4FC7
:102190000990D881C02DCE019464C9C0811540E555
:1021A000940708F069C0811550E4950708F060C0F5
:1021B0009A9581159F4108F4B9C0B5C0811536E5DF
:1021C000930728F5811545E5940708F092C081151D
:1021D00054E5950708F087C0AC0143705527282FB8
:1021E00026952695C115D34508F06CC081E090E096
:1021F00002C0880F991F4A95E2F740E2249F9001A0
:102200001124EC01C22BD32BCE019C6890C0811508
:102210002AE5920780F4811539E5930708F072C02A
:10222000811548E5940708F47EC0D82FCC27CE014D
:10223000806F906A7CC090568115904208F073C000
:102240008D2F8F710E944612DD27D0628F71AE01F3
:10225000582BCA016CC081E090E069C0C55AD0E03B
:10226000C059DE4F8881C82FD0E0CE0190645FC096
:10227000DF70CE01906A5BC074E0969587957A9581
:10228000E1F7282F23703C2F337081E090E002C0EB
:10229000880F991F3A95E2F79C68AC01522B9A017E
:1022A0009C2F9F709695969550E2959FE001112482
:1022B000C9018C2B9D2B3BC0D82FCC27CE01816F21
:1022C000906A35C081E090E002C0880F991F4A955E
:1022D000E2F750E2259F90011124EC01C22BD32B91
:1022E000CE019A6824C0D82FCC27CE01846F906A83
:1022F0001EC00E9446128F7190E0D82FCC27CE01CD
:10230000906215C08F700E94461294E0D695C795D2
:102310009A95E1F7CF70D0E0DC2FCC27D0699E01F1
:10232000282BC90104C080E090E001C0CE01DF91FC
:10233000CF91089526E6829FC0011124FC0121E17E
:10234000729FE00DF11D1124E60FF11DEE0FFF1F2E
:10235000E852FF4F8591949108950E949A110E942E
:10236000981008958238910569F1B0F48133910590
:1023700009F46DC048F48932910509F463C08A32CA
:10238000910509F469C008958533910509F455C094
:1023900089339105B9F00895833E910569F138F4C8
:1023A000803E9105B1F0823E910509F10895863E87
:1023B0009105A9F1873E9105B9F1843E910509F097
:1023C00064C023C02091730220FD4FC021FD4DC089
:1023D00008958091730280FD44C08091740280FF53
:1023E00044C08091730284FD42C083EE4DC0809151
:1023F000730282FF38C0F5CF8091730282FD33C033
:102400008091740280FD31C0ECCF8091740281FF15
:1024100032C08091730284FD2AC087EE35C080915E
:10242000730283FF26C0F5CF8091730283FD21C024
:102430008091740281FD1FC0ECCF8091730285FDF5
:102440001CC01DC08091730285FD19C016C080910B
:10245000730286FD16C017C08091730286FD13C0FB
:1024600010C089E311C082EE0FC080EE0DC080E085
:102470000BC086EE09C084EE07C089E205C085E383
:1024800003C08AE201C081E390E008959091730255
:1024900092FF0DC0282F2871283019F4877F84609F
:1024A00006C0282F2471243011F48B7F886093FF9D
:1024B0000DC0282F2871283119F4877E846106C049
:1024C000282F2471243111F48B7E886120917402AD
:1024D00020FF0DC0382F3871383019F4877F8160A4
:1024E00006C0382F3171313011F48E7F886021FFA2
:1024F0000DC0282F2871283119F4877E816106C00C
:10250000282F2171213111F48E7E886194FD877E00
:1025100008950C94D70E0E9404148FE39CE9019750
:10252000F1F700C000000E94041480E00E94C51270
:1025300060FF04C00E9489120C94A61808950C94A0
:102540008B120E94DD0E811102C00E94850F0E9435
:10255000E80E809353020E94F00E909374028093D1
:1025600073020E949F120E94EC0E682F70E080E0C0
:1025700090E00E94E5086091DF017091E001809198
:10258000E1019091E2010C941D0924E0829FC001B9
:102590001124FC01E357FD4F608171818281938199
:1025A0000895CF92DF92EF92FF920F931F93CF93F4
:1025B000DF938BEC92E00E946D028DE8E82E82E0C2
:1025C000F82EC0E0D0E096ECC92E92E0D92E0CEBAC
:1025D00012E0DF93CF93DF92CF920E94060383EC49
:1025E00092E00E946D02F701619171918191919148
:1025F0007F010E9413049F938F937F936F931F9388
:102600000F930E9406038AEB92E00E946D022196CE
:102610008DB79EB70A960FB6F8949EBF0FBE8DBFBA
:10262000C630D105B1F6DF91CF911F910F91FF9088
:10263000EF90DF90CF90089580EA8A95F1F70895A2
:1026400000C008950C941C1308950C9424130C944A
:1026500025130C9424130C942913F894E82FE29575
:10266000EF70F0E031A1282F2F7081E090E001C0E1
:10267000880F2A95EAF7982F9095932391A392A11A
:10268000892B82A3789408950F931F93CF93DF93A0
:10269000C4E8D1E089918F3F11F00E942D1381E0B1
:1026A000CA38D807B9F7C3E7D1E004E811E0899147
:1026B0008F3F11F00E942D130C171D07C1F7DF91FA
:1026C000CF911F910F9108954F925F926F927F92D9
:1026D0008F929F92AF92BF92DF92EF92FF920F93F1
:1026E0001F93CF93DF938C01C62FD0E0CE018C5780
:1026F0009E4F7C01FC0190819F3F09F460C0D62E63
:10270000F894E92FE295EF70F0E081A19F7021E04D
:1027100030E001C0220F9A95EAF7822B81A382A1B3
:102720002095282322A378940E942013E3E7F1E068
:1027300024E831E0412C512C32014394812C912C1E
:10274000540181918F3F99F0A82FA295AF70B0E00E
:1027500090964C9150E08F70BA0102C075956795C4
:102760008A95E2F760FD03C0D301C20103C080E097
:1027700090E0DC01882A992AAA2ABB2A440C551C1D
:10278000661C771C2E173F07E1F6F70180818F3F0B
:1027900011F00E942D1361E081149104A104B10491
:1027A00009F460E08D2D0E942213CC0FDD1FCC0FA9
:1027B000DD1FC00FD11F88829982AA82BB82DF9160
:1027C000CF911F910F91FF90EF90DF90BF90AF904E
:1027D0009F908F907F906F905F904F9008950E9490
:1027E000441388E1EDE8F2E0DF01982F1D929A95FD
:1027F000E9F7E5E7F2E0DF011D928A95E9F786E067
:102800000E944F140C946103FF920F931F93CF9378
:10281000DF93CDB7DEB768970FB6F894DEBF0FBE73
:10282000CDBF8E010F5F1F4F88E1F80111928A958D
:10283000E9F7F12C6F2DC8010E946413F394F6E0C0
:10284000FF12F8CF48E150E0B80185E792E00E941E
:102850004720FF24F394009709F4F12C892B41F0D1
:1028600088E1F801A5E7B2E001900D928A95E1F7C1
:102870002F2D46E06DE872E085E792E00E9450144B
:102880000E9463038F2D68960FB6F894DEBF0FBECB
:10289000CDBFDF91CF911F910F91FF9008950895C3
:1028A000FF920F931F93CF93DF93F82ED92F8B01B5
:1028B000C42F222349F081E0809356020E945918C8
:1028C0009093550280935402809156028823F1F030
:1028D00080915402909155020E9471180597B0F0B2
:1028E000EF2DFD2FD80180E090E04C2F50E08417B1
:1028F000950754F401911191219131910D931D93FC
:102900002D933D930196F3CF10925602DF91CF9114
:102910001F910F91FF9008950E94FB1A0E94C90F0A
:102920000C94071B0E940B1B0E9494100C94291BF3
:102930000E94F7170E94E21A0E94B70F0E948C149F
:102940000E9492140E94C10FFBCFCF93DF93EC0142
:10295000FB018281882309F43CC1C430FDE5DF0717
:1029600060F4CB3F9CE5D90788F49E0122503C459A
:102970002431310508F02EC109C0C236EDE5DE076D
:1029800029F0C63AFDE5DF0709F024C10E94F00EE8
:102990009093740280937302C1318CE5D80709F4D7
:1029A000C6C008F042C0C930ECE5DE0709F49BC0A0
:1029B00000F5C5308CE5D80709F485C078F4C3303C
:1029C000ECE5DE0709F478C008F07AC0C230DC45D7
:1029D00009F0F5C0809173028160EFC0C7309CE5BB
:1029E000D90709F478C008F07AC080917302806139
:1029F000E4C0CD30FCE5DF0709F487C058F4CB30E4
:102A00009CE5D90709F479C008F07BC08091730276
:102A100088606FC0CF30FCE5DF0709F480C008F0A4
:102A200082C080917302877FC8C0CE3F9CE5D907E2
:102A300009F471C000F5C531FCE5DF0709F485C074
:102A400068F4C3319CE5D90709F475C008F095C056
:102A50000E948D08809173028F77AFC0CC3FFCE558
:102A6000DF07A9F108F054C0CB3FDC4509F0A7C04F
:102A70008091740240C0C230EDE5DE0709F489C0E0
:102A800058F4C1158DE5D80709F45AC008F069C09B
:102A90008091740282602FC0C236EDE5DE0709F432
:102AA0007CC0C63AFDE5DF0709F481C0C330DD45CF
:102AB00009F085C080E06EC08091730282607DC0A5
:102AC0008091730216C080917302886076C08091F5
:102AD000740282604FC08091730280626EC08091E8
:102AE000730280646AC00E948D08809173028068BE
:102AF00064C0846062C081603DC0809173028E7F3B
:102B00005CC0809173028D7F58C08091730216C0A3
:102B10008091740218C0809174028D7F2BC08091C7
:102B200073028F7E4AC0809173028F7D46C0809170
:102B300073028F7B42C080917302877F8B7F3DC081
:102B4000809174028D7F8E7F15C08091730282FB0D
:102B5000222720F991E0922790FB82F990FB83F9DC
:102B60002CC080917402982F909591708E7F892B44
:102B700090FB81F98093740222C00E948D0880919D
:102B8000730287FB222720F991E0922790FB87F9B7
:102B900014C081E00E94870F12C08091730284FBF1
:102BA000222720F991E0922790FB84F906C08091BA
:102BB0007302982F909590FB80F980937302809117
:102BC0007302909174020E94010F0E948D0880E0B0
:102BD00001C081E0DF91CF910895CF93DF938631DB
:102BE0009C4541F5EB010E94E00D982F8A812091D0
:102BF000020130910301882379F09A7A81E009F487
:102C000080E080935702911102C069E201C065E340
:102C1000C9010E94B0170AC080915702811102C0F9
:102C200069E201C065E3C9010E94B2170E94220E49
:102C300080E001C081E0DF91CF9108950F931F9351
:102C4000CF93DF93C42FD22FFC0182818823C9F058
:102C500040935A020E945918909359028093580247
:102C600080E28C0F883008F057C0C77081E001C047
:102C7000880FCA95EAF7DF91CF911F910F910C94BD
:102C8000F90580915A02481330C080915802909102
:102C900059020E947118883C910538F510E21D0F09
:102CA000CD17B9F080E28C0F883040F4C77081E016
:102CB00001C0880FCA95EAF70E940006183028F56F
:102CC00081E09D2F977001C0880F9A95EAF70E94C6
:102CD000F905802F0E94F0051830F0F4D77081E0DC
:102CE00001C0880FDA95EAF70AC080E28C0F8830BD
:102CF00098F4C77081E001C0880FCA95EAF7DF91A8
:102D0000CF911F910F910C940006802FDF91CF91EE
:102D10001F910F910C94F005DF91CF911F910F91AE
:102D200008950F939C01CB01243F4CE5340731F10A
:102D300088F4293DFCE53F07D9F02A3D4CE53407EE
:102D400079F1283D3C45A9F506E221EE41EE68ED1A
:102D50007CE52BC0263FFCE53F07E1F0A8F0273FCC
:102D60003C4539F507E225EE46EE67EF7CE51DC0F0
:102D700007E225EE45EE69ED7CE517C006E221EE9F
:102D800040EE64EF7CE511C007E225EE44EE65EF0E
:102D90007CE50BC006E221EE42EE66EF7CE505C065
:102DA00008E221E045EE6AED7CE50E941E1680E017
:102DB00008C0FC018281882319F010925A0201C0D8
:102DC00081E00F91089590939B0180939A0108955B
:102DD0009093600280935F020895E0915F02F0910A
:102DE0006002309721F00190F081E02D099480E09D
:102DF0000895EF92FF920F931F93CF93DF93E0918B
:102E00005F02F09160023097B1F18C010280F38192
:102E1000E02D09958091530282FF2DC080FF04C0F0
:102E20008AEF92E00E946D02E80118E084EFE82E3C
:102E300082E0F82E8091530280FF0BC088811F92A0
:102E40008F93FF92EF920E9406030F900F900F90C6
:102E50000F90115021961111EDCF8091530280FFF8
:102E60000AC082EF92E0DF91CF911F910F91FF9006
:102E7000EF900C946D02DF91CF911F910F91FF9015
:102E8000EF90089520915D0230915E022817390776
:102E900071F090935E0280935D02E0915F02F09189
:102EA0006002309721F00680F781E02D09940895A3
:102EB00020915B0230915C022817390771F09093E2
:102EC0005C0280935B02E0915F02F09160023097B8
:102ED00021F00084F185E02D09940895FC013296DB
:102EE00097E080E0915029F021912223D9F38F5F60
:102EF000F9CF0895662349F0FC0132960896219196
:102F0000621729F0E817F907D1F780E0089581E00A
:102F100008959C01FC0132969FEF80E04191461795
:102F200089F09F3F19F4411101C0982F8F5F8630BF
:102F3000A9F79F3F39F0F901E90FF11D97FDFA95C7
:102F40006283089508959C012A5F3F4FFC014281EE
:102F5000461301C01282019682179307B9F70895AC
:102F60000C9489170C94A317029626E0FC01119289
:102F70002A95E9F7089508950C94BB1783E0809390
:102F800061020C94BC17811102C081E001C082E093
:102F9000809361020C94BC170C94C31781E080935A
:102FA00061020C94BC170C94CE1708950C94D5179D
:102FB0000C94D6170C94D5170C94D5170C94D517E0
:102FC000CF930E94DC170E9404140E94DA17C0E01D
:102FD0008C2F0E94C512672B682B692B29F4CF5FB9
:102FE000C630B1F780E001C081E0CF910895089527
:102FF0001F920F920FB60F9211248F939F93AF934E
:10300000BF9380916202811113C08091A5029091BB
:10301000A602A091A702B091A8024196A11DB11DE0
:103020008093A5029093A602A093A702B093A80252
:10303000BF91AF919F918F910F900FBE0F901F90F6
:1030400018958091AD02843031F10E94E603109210
:10305000620220E488E190E00FB6F894A89580938E
:1030600060000FBE2093600083B7817F846083BFC0
:1030700083B7816083BF7894889583B78E7F83BF41
:103080000FB6F894A89580916000886180936000E5
:10309000109260000FBE08950E948D080C94EA0300
:1030A00082E084BD93E095BD9AEF97BD80936E005A
:1030B00008952FB7F8948091A5029091A602A0914F
:1030C000A702B091A8022FBF08952FB7F89460917E
:1030D000A5027091A6028091A7029091A8022FBF2D
:1030E00008959C014FB7F8948091A5029091A60293
:1030F000A091A702B091A8024FBF821B930B089525
:1031000078941F920F920FB60F9211248F939F9372
:10311000AF93BF938091A5029091A602A091A702C0
:10312000B091A8020196A11DB11D8093A5029093B4
:10313000A602A093A702B093A802BF91AF919F915E
:103140008F910F900FBE0F901F90189581E0809384
:10315000E00080E28093D8001092C9008FE19EE4E5
:103160000197F1F700C0000087E090EBDC0180934D
:10317000B6029093B702A093B802B093B9029CE054
:1031800088E10FB6F894A895809360000FBE9093E5
:103190006000FFCF8091710208950895CF93DF936F
:1031A00021E02093E9002FEF3091E800215035FD18
:1031B00006C035ED3A95F1F700002111F5CF2091C9
:1031C000E80025FF14C0EC0140E050E068E070E04A
:1031D0000E94981B8091E8008E778093E80088E039
:1031E000FE01A9E6B2E001900D928A95E1F7DF9128
:1031F000CF91089580936502709367026093660291
:103200008091AD02843001F582E08093E9008FEF78
:103210009091E800815095FD06C095ED9A95F1F7E3
:1032200000008111F5CF8091E80085FF0DC040E0DE
:1032300050E063E070E085E692E00E94981B809188
:10324000E8008E778093E8000895BC0184E00C9438
:10325000FA18BC0183E00C94FA18089580E293E018
:103260000E946D028091AC02811109C00E94291D4B
:103270000E94861D8091E20084608093E2000895A0
:103280008CE193E00E946D021092AC02089588E1F7
:1032900093E00E946D020C94D31784E193E00E94A6
:1032A0006D026091A90281E0611101C080E00C947F
:1032B000BE1780E193E00E946D029091AD0281E023
:1032C000943009F080E06091A9020C94C31720911A
:1032D00064022F5F822F62E30E943520992319F048
:1032E00020936402089510926402809168028823FA
:1032F00071F18091AD02843041F58091E9008F70C9
:103300002091EC00922F917020FD90E8892B93E0A2
:103310009093E9009091EB0090FF14C09091EE0023
:1033200097FF10C09091E80095FF03C01092F10044
:10333000F9CF9091E80090FF05C09091E8009E774A
:103340009093E8008F708093E900109268020895CE
:1033500042E061EC81E00E94A21C42E261EC82E06A
:103360000E94A21C42E261EC83E00E94A21C9091A8
:10337000AD0281E0943009F080E06091A9020C94E4
:10338000CC178091AF02833009F461C030F48130F2
:1033900071F0823009F49AC008958A3009F486C029
:1033A0008B3009F46CC0893009F0A8C020C080912E
:1033B000AE02813A09F0A2C08091E800877F809335
:1033C000E8008091B2029091B302892B21F468E069
:1033D00089E692E003C060E080E090E070E00E9447
:1033E000E31B8091E8008B778093E800089580913B
:1033F000AE02813209F082C08091B2029091B30294
:10340000029708F07BC08091E800877F8093E800F6
:103410008091E80082FD05C08091AD028111F8CF56
:103420006DC02091F3008091F20090E0922B029702
:1034300031F48091F100813011F0863021F48091D7
:10344000F100809371028091E8008B7753C08091E6
:10345000AE02813A09F052C08091B2029091B3025B
:10346000892B09F04BC08091E800877F8093E800AA
:103470008091E80080FFFCCF8091100136C08091E0
:10348000AE028132D9F58091B2029091B302892BBC
:10349000A9F58091E800877F8093E8000E94D71CFF
:1034A0008091B002809310010C948D088091AE023F
:1034B000813221F58091E800877F8093E8000E94A7
:1034C000D71C8091B1028093720208958091AE0260
:1034D000813AA1F48091E800877F8093E800809191
:1034E000E80080FFFCCF809172028093F100809110
:1034F000E8008E778093E8000C94D71C08959FB75E
:10350000F894109268029FBF9091AD02943009F038
:1035100057C09091E9009F703091EC00232F2170EB
:1035200030FD20E8922B23E02093E9002091EB006E
:1035300020FF43C02091EE0027FF3FC0209163028F
:10354000222321F02091E80025FF37C0109263026A
:1035500026E03091E80035FD15C03091AD023430E1
:1035600061F53091EB0035FD28C0215021F481E058
:103570008093630222C0EFE9FFE03197F1F700C0CA
:103580000000E7CF8093F1008091E80085FD0AC03C
:103590008091E80080FFFCCF8091E8008E778093D7
:1035A000E80006C08FB7F89421E0209368028FBF2F
:1035B0009F709093E90080E008959F709093E900D8
:1035C0008FEF089584B7877F84BF0FB6F894A895CE
:1035D00080916000886180936000109260000FBE4F
:1035E00090E080E80FB6F8948093610090936100BA
:1035F0000FBE0C94CE170E94291D0E94861DE2EE7C
:10360000F0E080818460808378940C941A2084E0B8
:1036100091E00C94E8168091AD028530C9F48CE0FD
:1036200093E00E946D028091AD02853079F40E9492
:1036300021188091AB028823B1F30E94E017882300
:1036400091F30E94821B0E948D08EDCF0C944C18C0
:10365000089508950C942C1B292F3327233031050E
:10366000C9F060F42130310581F02230310509F0D4
:1036700041C08BE590E02CE433E040C021323105BD
:10368000E1F02232310531F135C082E190E027EAE4
:1036900033E034C099278130910549F028F0029732
:1036A00049F5E4E2F3E005C0E8E4F3E002C0E8E352
:1036B000F3E0849190E09F0121C063307105D0F464
:1036C000660F771FFB01ED56FE4F2081318189E0A7
:1036D00090E014C06330710568F4FB01EE0FFF1F2A
:1036E000E357FE4F20813181FB01E657FE4F808179
:1036F00090E004C080E090E020E030E0FA01318307
:103700002083089580E189BD82E189BD09B400FE6E
:10371000FDCF8091D8008F7D8093D8008091E0000C
:1037200082608093E0008091E00081FDFCCF0895ED
:10373000CF92DF92EF92FF920F931F93CF93DF937D
:10374000EC018B017A010E94F61C811133C0E11457
:10375000F10439F0F70180819181081B190BC80F22
:10376000D91FC12CD12C0115110519F18091E80048
:1037700085FD16C08091E8008E778093E800E11403
:10378000F10449F0F70180819181C80ED91ED182E0
:10379000C08285E00FC00E94F61C882321F30AC076
:1037A00089918093F10001501109FFEFCF1ADF0AD0
:1037B000DACF80E0DF91CF911F910F91FF90EF90D2
:1037C000DF90CF9008952091B4023091B502261772
:1037D000370748F06115710539F42091E8002E771C
:1037E0002093E80001C0B901FC0120E061157105DA
:1037F00079F18091AD028823F1F18530F1F180916A
:10380000E80083FD3CC08091E80082FD2EC08091DD
:10381000E80080FFEBCF2091F3008091F20090E070
:10382000922B6115710551F08830910538F4219182
:103830002093F100615071090196F3CF21E00897C0
:1038400009F020E08091E8008E778093E800CECFE9
:103850002111CFCF0AC08091AD02882361F085305D
:1038600061F08091E80083FD0AC08091E80082FF4A
:10387000F2CF80E0089582E0089583E0089581E02A
:1038800008952091B4023091B5022617370748F009
:103890006115710539F42091E8002E772093E80036
:1038A00001C0B901FC0120E06115710591F1809121
:1038B000AD02882309F440C0853009F43FC08091EF
:1038C000E80083FD3DC08091E80082FD2FC080911B
:1038D000E80080FFE9CF2091F3008091F20090E0B2
:1038E000922B6115710559F08830910540F42491AF
:1038F0002093F1003196615071090196F2CF21E0D9
:10390000089709F020E08091E8008E778093E80026
:10391000CBCF2111CCCF0AC08091AD02882361F0BA
:10392000853061F08091E80083FD0AC08091E80055
:1039300082FFF2CF80E0089582E0089583E0089549
:1039400081E00895982F973068F59093E9009817D3
:1039500039F07091EC002091ED005091F00003C01F
:10396000242F762F50E021FD02C09F5FECCF3091D5
:10397000EB003E7F3093EB003091ED003D7F3093C4
:10398000ED003091EB0031603093EB007093EC0070
:103990002093ED005093F0002091EE0027FDE5CF3D
:1039A00080E008958F708093E90081E00895809110
:1039B000AE0287FF11C08091E80082FD05C08091B2
:1039C000AD028111F8CF11C08091E8008B770BC058
:1039D0008091AD02882349F08091E80080FFF8CF04
:1039E0008091E8008E778093E80008952091E400AC
:1039F0003091E50095E64091EC00842F817040FF06
:103A000023C08091E80080FD1DC08091AD02882315
:103A100099F0853099F08091EB0085FD11C04091BF
:103A2000E4005091E5002417350729F3915011F077
:103A30009A01E1CF84E0089582E0089583E008953B
:103A400081E0089580E008954091E80042FFDDCFD5
:103A500008950E94971D0E949F1DE0EEF0E0808176
:103A600081608083E8EDF0E080818F77808319BCEE
:103A7000A7EDB0E08C918E7F8C9380818F7E8083C8
:103A80001092AC0208950F931F93CF93DF930E947F
:103A9000971D0E949F1DC8EDD0E088818F77888395
:103AA00088818068888388818F7D888319BC109283
:103AB000AD021092A9021092AB021092AA0200EE7F
:103AC00010E0F80180818B7F80838881816088830A
:103AD00042E060E080E00E94A21CE1EEF0E0808124
:103AE0008E7F8083E2EEF0E0808181608083808140
:103AF00088608083F80180818E7F808388818061E7
:103B00008883DF91CF911F910F910895E8EDF0E048
:103B100080818F7E8083E7EDF0E08081816080830B
:103B200084E082BF81E08093AC020C94431DE8EDF9
:103B3000F0E080818E7F80831092E20008951092E1
:103B4000DA001092E10008951F920F920FB60F92C3
:103B500011242F933F934F935F936F937F938F9392
:103B60009F93AF93BF93EF93FF938091E10082FF08
:103B70000BC08091E20082FF07C08091E1008B7F43
:103B80008093E1000E9467198091DA0080FF1FC0D6
:103B90008091D80080FF1BC08091DA008E7F8093D7
:103BA000DA008091D90080FF0DC080E189BD82E1FB
:103BB00089BD09B400FEFDCF81E08093AD020E9473
:103BC0002E1905C019BC1092AD020E9440198091B7
:103BD000E10080FF19C08091E20080FF15C0809154
:103BE000E2008E7F8093E2008091E200806180930A
:103BF000E2008091D80080628093D80019BC85E0F3
:103C00008093AD020E944D198091E10084FF30C085
:103C10008091E20084FF2CC080E189BD82E189BDF2
:103C200009B400FEFDCF8091D8008F7D8093D8002D
:103C30008091E1008F7E8093E1008091E2008F7E91
:103C40008093E2008091E20081608093E2008091A5
:103C5000A902882311F084E007C08091E30087FD6A
:103C600002C081E001C083E08093AD020E94591937
:103C70008091E10083FF29C08091E20083FF25C08D
:103C80008091E100877F8093E10082E08093AD0224
:103C90001092A9028091E1008E7F8093E1008091D3
:103CA000E2008E7F8093E2008091E2008061809349
:103CB000E20042E060E080E00E94A21C8091F000FF
:103CC00088608093F0000E944719FF91EF91BF91A7
:103CD000AF919F918F917F916F915F914F913F91A4
:103CE0002F910F900FBE0F901F9018951F920F925B
:103CF0000FB60F9211242F933F934F935F936F93BF
:103D00007F938F939F93AF93BF93CF93DF93EF9363
:103D1000FF93C091E900CF708091EC00D82FD17053
:103D200080FDD0E81092E9008091F000877F8093B9
:103D3000F00078940E94BA1E1092E9008091F00081
:103D400088608093F000CD2BCF70C093E900FF9185
:103D5000EF91DF91CF91BF91AF919F918F917F9123
:103D60006F915F914F913F912F910F900FBE0F90E8
:103D70001F9018951F93CF93DF93CDB7DEB7AA9707
:103D80000FB6F894DEBF0FBECDBFEEEAF2E0809131
:103D9000F100819322E0E63BF207C9F70E94C119C6
:103DA0008091E80083FF2EC18091AE029091AF0216
:103DB000492F50E04A30510508F024C1FA01EE596C
:103DC000FF4F0C944120803821F0823809F01AC14D
:103DD00008C08091AA029091AB02992389F0826079
:103DE0000FC08091B2028F70873008F00BC18093B2
:103DF000E9008091EB0085FB882780F91092E900AB
:103E00009091E800977F9093E8008093F1001092E2
:103E1000F100D1C0282F2D7F09F0F4C0882319F0BC
:103E2000823061F0EFC08091B002813009F0EAC0C9
:103E3000933009F080E08093AB022EC08091B002F5
:103E400081112AC08091B2028F702FEF280F263087
:103E500008F0D8C08093E9002091EB0020FF1CC03F
:103E6000933021F48091EB00806214C09091EB00BC
:103E700090619093EB0021E030E0A90102C0440F73
:103E8000551F8A95E2F74093EA001092EA0080916C
:103E9000EB0088608093EB001092E9008091E800CD
:103EA000877F8093E8000E94D71CACC08111AAC014
:103EB0001091B0021F778091E3008078812B80936E
:103EC000E3008091E800877F8093E8000E94D71C80
:103ED0008091E80080FFFCCF8091E30080688093B0
:103EE000E300111102C082E001C083E08093AD02C3
:103EF00089C08058823008F085C08091B0029091CE
:103F0000B1028C3D53E0950779F583E08A838AE21C
:103F100089834FB7F894DE01139620E03EE051E22A
:103F2000E32FF0E050935700E49120FF03C0E295A7
:103F3000EF703F5FEF708E2F90E0EA3010F0C79681
:103F400001C0C0968D939D932F5F243149F74FBFD9
:103F50008091E800877F8093E8006AE270E0CE01FC
:103F600001960E94E31B16C06091B2027091B302E9
:103F7000AE014F5F5F4F0E942A1BBC01892B09F4E1
:103F800041C09091E800977F9093E80089819A81E1
:103F90000E94411C8091E8008B778093E80032C03A
:103FA000803881F58091E800877F8093E8008091D8
:103FB000A9028093F1008091E8008E7772CF811181
:103FC00021C08091B0029091B10299270297D4F458
:103FD0008091E800877F8093E8008091B002809311
:103FE000A9020E94D71C8091A902811106C080916C
:103FF000E30087FD02C081E001C084E08093AD0250
:104000000E94A8198091E80083FF0AC08091E8000F
:10401000877F8093E8008091EB0080628093EB00C3
:10402000AA960FB6F894DEBF0FBECDBFDF91CF9139
:104030001F910895CF938091AD028823A1F0C09184
:10404000E900CF709091EC00892F817090FD80E89D
:10405000C82B1092E9008091E80083FD0E94BA1EEF
:10406000CF70C093E900CF910895991B79E004C007
:10407000991F961708F0961B881F7A95C9F78095A7
:104080000895EE0FFF1F0590F491E02D0994FB01B8
:10409000DC0104C08D910190801921F44150504001
:1040A000C8F7881B990B0895F999FECF92BD81BD81
:1040B000F89A992780B50895A8E1B0E042E050E071
:1040C0000C948820262FF999FECF92BD81BDF89AD5
:1040D000019700B4021639F01FBA20BD0FB6F8944C
:1040E000FA9AF99A0FBE08950396272F0E9463202B
:1040F0000E946220252F0E946320242F0C946320AD
:104100000196272F0E9463200C946220DC01CB01D2
:10411000FC01F999FECF06C0F2BDE1BDF89A3196D7
:1041200000B40D9241505040B8F70895F894FFCF75
:10413000C8002902CA18CE182D1929192519CD1819
:1041400001E200E900EA00B500B600B700CD008347
:1041500001CC008A0192019401210223022402254C
:1041600002260227022A02B300B4006F0070008109
:104170008283E200E900EA00B500B600B700CD0096
:104180008301CC008A0192019401210223022402BE
:104190002502260227022A02B300B4006F00700035
:1041A000818283F067F166F436F535F634F7979639
:1041B000953331329091929394374032220D04DB43
:0A41C00003B9035E037703900300C8
:00000001FF
